:020000040800F2
:10000000E0070020BD250008590300085B03000835
:100010005F03000863030008670300080000000096
:100020000000000000000000000000006B0300085A
:100030006D030008000000006F0300087103000852
:10004000D7250008D7250008D7250008D7250008A0
:10005000D7250008D7250008D7250008D725000890
:10006000D7250008D7250008D7250008D725000880
:10007000D7250008D7250008D7250008D725000870
:10008000D7250008D7250008D7250008D725000860
:10009000D7250008D7250008D7250008D725000850
:1000A000D7250008D7250008D7250008D725000840
:1000B000D7250008232700085D270008D72500085A
:1000C000D7250008D7250008D7250008D725000820
:1000D000D7250008333200084B3200088932000867
:1000E000D7250008D7250008D725000800F002F81A
:1000F00000F062F80AA090E8000C82448344AAF160
:100100000107DA4501D100F057F8AFF2090EBAE85D
:100110000F0013F0010F18BFFB1A43F0010318473B
:10012000203B0000403B0000103A24BF78C878C153
:10013000FAD8520724BF30C830C144BF04680C60ED
:10014000704700000023002400250026103A28BF35
:1001500078C1FBD8520728BF30C148BF0B60704739
:10016000692903F02F81642903F02C81752903F09C
:1001700029816F2903F0C081782903F0E7810368A2
:10018000DB0928BF41F08001632903F0FC83732958
:1001900003F00184E32903F01F84002070471FB59A
:1001A00003F078FC04000020002103F0C9FC401C8F
:1001B00060601FBD10B510BD03F046FC1146FFF78F
:1001C000EEFF00F067F803F069FC03B4FFF7F2FFFD
:1001D00003BC02F0F1FE000010B54DA003F070F872
:1001E0004FF4967002F0B5FE4BA14C4803F09EFA16
:1001F000044647A003F064F84FF4967002F0A9FE9D
:1002000045A1464803F092FA044602F02DFAC4B91B
:100210000120434908604FF4967002F09AFE4FF4B3
:10022000967002F096FE4FF4967002F092FE4FF434
:10023000967002F08EFE00203A49C1F8800102F06B
:1002400013FA33A003F03CF84FF4967002F081FEED
:1002500002F00AFA30A1314803F068FA044632A0ED
:1002600003F02EF84FF4967002F073FE002031492F
:10027000086002F0F9F930A003F022F84FF496700C
:1002800002F067FE30A003F01BF84FF4967002F006
:1002900060FE10BD1CB502F01FFE02F087FE02F0EA
:1002A000ADF94FF4E13002F0B1FE4FF4E13002F06D
:1002B000FCFE40F27121072002F0C4F900BF02F0F9
:1002C000ECFD0028FBD1FFF787FF02F06EFA02F089
:1002D00079FB1BE0694601A802F0B3FD20200190E4
:1002E000432000909DF800109DF8040002F0C6FB2A
:1002F0004FF4FA7002F02DFE0E48006808B9012094
:1003000000E000200B49086002F0AEF9E2E70000CF
:1003100041540D0A000000004F4B0000B7000020C0
:1003200080012142000021424154453026570D0AE8
:10033000000000008081214241542B514D5444491A
:1003400053433D300D0A000041542B514D54434C52
:100350004F53453D300D0A00704700BFFEE700BF18
:10036000FEE700BFFEE700BFFEE77047704770473B
:100370007047000010B500F03DFE012000F0BFFE08
:1003800000BF212000F079FE0028FAD0102000F0F4
:1003900099F9022000F082F9002000F0D0FE002040
:1003A00000F0DFFE4FF4806000F0D2FE4FF46011E9
:1003B000002000F0A7FE012000F0B0FE00BF3920B1
:1003C00000F05BFE0028FAD0022000F0AAFE00BF79
:1003D00000F0B0FE0828FBD101211D2000F078FFBD
:1003E00010BD0CB50020019000906C48006840F4EE
:1003F00080306A49086000BF6848006800F4003037
:1004000000900198401C0190009818B90198B0F52F
:10041000A06FF1D16148006800F4003010B10120F4
:10042000009001E0002000900098012843D15C4832
:10043000006840F010005A4908600846006820F043
:10044000030008600846006840F002000860534856
:10045000406852494860084640684860084640681D
:1004600040F4806048600846406820F47C10486092
:100470000846406840F4E81048600846006840F0CC
:100480008070086000BF4548006800F000700028D8
:10049000F9D04248406820F00300404948600846CF
:1004A000406840F00200486000BF3C48406800F0EF
:1004B0000C000828F9D10CBD10B5FFF792FF10BD54
:1004C00010B53648006840F001003449086008461D
:1004D000406834490840314948600846006832495C
:1004E00008402E4908600846006820F48020086013
:1004F0000846406820F4FE0048604FF41F00886002
:10050000FFF7DAFF4FF000602849086010BD10B512
:10051000002100200022214B5B6803F00C0121B177
:10052000042906D0082928D107E0214B214C23605B
:1005300027E01F4B1F4C236023E0184B5B6803F43C
:100540007010164B5B6803F48032022303EB90407B
:1005500022B9194B4343174C23600DE00F4B5B68E6
:1005600003F4003323B1144B4343124C236003E0E4
:100570000F4B43430F4C236003E00D4B0D4C2360A6
:1005800000BF00BF054B5B68C3F303130B4CE15C7A
:10059000084B1B68CB40074C236010BD0010024085
:1005A000002002400000FFF8FFFFF6FE08ED00E02B
:1005B00000127A000000002000093D000400002025
:1005C00031490143314A1160704770B50021002361
:1005D0000F22C47804B32D4C246804F4E064C4F5FD
:1005E000E064210AC1F10403CA40447804FA03F12B
:1005F0008478144021430901254C0678A1550478DC
:1006000004F01F050124AC4005786D11AD0005F123
:10061000E025C5F8004109E0047804F01F05012435
:10062000AC401C4D0678761145F8264070BD1A4A3C
:100630000A400243154B1B1F1A60704739B1134A19
:10064000121D12680243114B1B1D1A6006E00F4A6F
:10065000121D126882430D4B1B1D1A60704704283F
:1006600008D14FF0E021096941F004014FF0E02288
:10067000116107E04FF0E021096921F004014FF01A
:10068000E0221161704700000000FA050CED00E067
:1006900000E400E080E100E080FFFF1F0146002051
:1006A000FE4A106800F03800084310607047FB49AC
:1006B000096821F00801F94A1160114609680143EF
:1006C00011607047F549096821F01001F34A116083
:1006D00011460968014311607047F148EF494860CD
:1006E000F04848607047EE48EC494860ED48486083
:1006F0007047EA48006940F08000E84908617047A7
:10070000E648006940F08000E44908617047042031
:10071000E249C96801F0010109B101200EE0DF4999
:10072000C96801F0040109B1022007E0DB49C9688A
:1007300001F0100109B1032000E00420704700B56A
:1007400002460423FFF7E3FF034603E0FFF7DFFF62
:100750000346521E012B01D1002AF7D102B905230D
:10076000184600BD30B5044604254FF43020FFF78D
:10077000E6FF0546042D17D1C848006940F0020085
:10078000C649086108464461006940F040000861BC
:100790004FF43020FFF7D3FF0546C048006941F60B
:1007A000FD710840BD490861284630BD10B50424DC
:1007B0004FF43020FFF7C3FF0446042C16D1B7488E
:1007C000006940F00400B54908610846006940F03E
:1007D000400008614FF43020FFF7B1FF0446AF48F6
:1007E000006941F6FB710840AC490861204610BD24
:1007F00000B502460423FFF78AFF034603E0FFF734
:1008000086FF0346521E012B01D1002AF7D102B9FF
:100810000523184600BD10B504244FF43020FFF71F
:10082000E7FF0446042C16D19C48006940F0040000
:100830009A4908610846006940F0400008614FF499
:100840003020FFF7D5FF04469448006941F6FB715C
:10085000084092490861204610BD00208F49C969AF
:1008600001F0020109B1012000E00020704730B51D
:10087000A5250424FFF7F1FF00B100254FF4302037
:10088000FFF75DFF0446042C3AD185488349886010
:10089000844888600846006940F0200008610846E6
:1008A000006940F0400008614FF43020FFF747FF37
:1008B0000446042C1BD17948006941F6DF710840D9
:1008C000764908610846006940F0100008617648E2
:1008D0000580E002FFF733FF0446052C10D06F4877
:1008E000006941F6EF7108406C49086108E0052C89
:1008F00006D06A48006941F6EF710840674908610F
:10090000204630BD78B506460C46042500200090F0
:10091000E802FFF714FF0546042D24D15F48006963
:1009200040F001005D4908613480E802FFF707FFED
:100930000546042D10D1B01C0090200C00990880B1
:10094000E802FFF7FCFE05465448006941F6FE71D7
:1009500008405249086106E05048006941F6FE71BE
:1009600008404E490861284678BD70B504460D46DA
:100970000426F002FFF7E3FE0646042E11D1474895
:10098000006940F00100454908612580F002FFF749
:10099000D6FE06464148006941F6FE7108403F49CF
:1009A0000861304670BD70B505460E460424E0026D
:1009B000FFF7C5FE0446042C17D139483749886033
:1009C000384888600846006940F0100008612E80B1
:1009D000E002FFF7B4FE0446052C06D02F4800695C
:1009E00041F6EF7108402D490861204670BD2DE9A0
:1009F000F04304464FF6FF763746B046B14604252D
:100A0000E443E6B2C4F30727C4F307484FEA146986
:100A1000E802FFF794FE0546042D49D120481F49FE
:100A20008860204888600846006940F0100008612E
:100A3000FF2E06D01C4808300680E802FFF77FFE34
:100A40000546042D08D1FF2F06D017480A3007802D
:100A5000E802FFF774FE0546042D0AD1B8F1FF0F36
:100A600007D011480C30A0F80080E802FFF767FEBD
:100A70000546042D0AD1B9F1FF0F07D00A480E3000
:100A8000A0F80090E802FFF75AFE0546052D0FD0AA
:100A90000248006941F6EF71084007E0002002407B
:100AA00023016745AB89EFCD00F8FF1F6649086158
:100AB0002846BDE8F08330B5054604244FF43020C5
:100AC000FFF73DFE0446042C41D160485E49886032
:100AD0005F4888600846006940F0200008610846C9
:100AE000006940F0400008614FF43020FFF727FE16
:100AF0000446042C22D15448006941F6DF710840B5
:100B0000514908610846006940F0100008611DB1B4
:100B100000205049088002E0A5204E4908804FF48B
:100B20003020FFF70CFE0446052C10D04648006923
:100B300041F6EF7108404449086108E0052C06D0F1
:100B40004148006941F6DF7108403F49086120468D
:100B500030BDF0B505460E46174604243B483A49D9
:100B600088603B488860E002FFF7E9FD0446042CFA
:100B700019D13548006940F010003349086147F049
:100B8000F800304328433349891C0880E002FFF70E
:100B9000D6FD0446052C06D02B48006941F6EF71BE
:100BA0000840294908612046F0BD2748C0698008EF
:100BB00070472548006A704700202349096801F002
:100BC000200109B1012000E00020704729B11E4A30
:100BD000126902431C4B1A6104E01B4A12698243EA
:100BE000194B1A61704701460020012908D1164AA5
:100BF000D26902F001020AB1012008E0002006E0FB
:100C0000114AD2680A400AB1012000E00020704772
:100C10000D49C860704704200B49C96801F0010103
:100C200009B101200EE00849C96801F0040109B1C9
:100C3000022007E00449C96801F0100109B103204E
:100C400000E00420704700000020024023016745B7
:100C5000AB89EFCD00F8FF1F10B50446CC488442A5
:100C600008D10121042000F04DFB0021042000F0F8
:100C700049FB46E0C748844208D10121082000F022
:100C800041FB0021082000F03DFB3AE0C2488442CD
:100C900008D10121102000F035FB0021102000F0C8
:100CA00031FB2EE0BD48844208D10121202000F014
:100CB00029FB0021202000F025FB22E0B8488442D7
:100CC00008D10121402000F01DFB0021402000F050
:100CD00019FB16E0B348844208D10121802000F0BE
:100CE00011FB0021802000F00DFB0AE0AE48844299
:100CF00007D10121801500F005FB0021A01500F0AF
:100D000001FB10BD10B50121084600F0FBFA0021DF
:100D1000012000F0F7FA10BD2DE9F0410246002550
:100D20000026002000230024002791F803C00CF0C7
:100D30000F0591F803C00CF0100CBCF1000F03D0AC
:100D400091F802C04CEA050591F800C0BCF1000F13
:100D500031D0146800202BE04FF0010C0CFA00F3A6
:100D6000B1F800C00CEA03069E4220D183004FF088
:100D70000F0C0CFA03F7BC4305FA03FC4CEA04041D
:100D800091F803C0BCF1280F06D14FF0010C0CFA0A
:100D900000FCC2F814C00AE091F803C0BCF1480F8F
:100DA00005D14FF0010C0CFA00FCC2F810C0401C39
:100DB0000828D1D31460B1F800C0BCF1FF0F34DDB6
:100DC000546800202EE000F1080C4FF0010808FAEA
:100DD0000CF3B1F800C00CEA03069E4221D1830057
:100DE0004FF00F0C0CFA03F7BC4305FA03FC4CEA76
:100DF000040491F803C0BCF1280F05D100F1080CE0
:100E000008FA0CF8C2F8148091F803C0BCF1480F3E
:100E100007D100F1080C4FF0010808FA0CF8C2F8ED
:100E20001080401C0828CED35460BDE8F0814FF6F6
:100E3000FF710180022181700421C1707047024658
:100E4000002093680B400BB1012000E000207047A8
:100E50000146886880B2704702460020D3680B4084
:100E60000BB1012000E0002070470146C86880B245
:100E7000704701617047416170470AB1016100E04C
:100E800041617047C16070474FF480320A4382610C
:100E90008161826182698269704702460020434B0A
:100EA00018684FF68073184040EA021008433F4B21
:100EB000186070473E49C8617047F0B50A46002384
:100EC00000240021002500F00046B6F1004F02D1B9
:100ED000364EF16901E0354E7168C0F3034583B2C7
:100EE00000F44016B6F5401F08D121F070612F4E76
:100EF000766826F070662D4F7E6012E000F4801652
:100F0000B6F5801F06D1032606FA05F4A14341F089
:100F1000706106E0460D360103FA06F6B14341F072
:100F2000706122B1460D360103FA06F6314300F036
:100F30000046B6F1004F02D11C4EF16101E01B4E9C
:100F40007160F0BD30B500228B071C0F0F2303FA30
:100F500004F2164B08338C1053F824309343134C8F
:100F600008348D1044F8253023468C1053F8243073
:100F70008C07240F00FA04F423430C4C08348D1022
:100F800044F8253030BD0A49DC3108607047000064
:100F900000080140000C0140001001400014014015
:100FA00000180140001C01400020014000000140E9
:100FB000000020420E49086070470D4948607047A4
:100FC0000B49886070474AF6AA20094908607047B3
:100FD0004CF6CC4006490860704701460020044AA0
:100FE000D2680A400AB1012000E0002070470000EA
:100FF00000300040DF48006840F00100DD49086033
:1010000008464068DC490840DA49486008460068FC
:10101000DA490840D74908600846006820F4802073
:1010200008600846406820F4FE0048604FF41F0046
:1010300088607047CF49096821F48031CD4A11603A
:101040001146096821F480211160B0F5803F03D07A
:10105000B0F5802F0ED106E0C649096841F4803111
:10106000C44A116007E0C349096841F4A021C14A9C
:10107000116000E000BF00BF704710B501460022BC
:10108000002300204A11012A02D1BA4C236806E04D
:10109000022A02D1B74C236A01E0B64C636A01F020
:1010A0001F02012494401C400CB1012000E00020EC
:1010B00010BD38B5002000900024002500BF31206D
:1010C000FFF7DBFF05460098401C00900098B0F544
:1010D000A06F01D0002DF2D03120FFF7CEFF08B174
:1010E000012400E00024204638BD01460020A14A2A
:1010F000106820F0F80040EAC10010607047A04975
:1011000008607047024600209A4B586820F47C1013
:1011100042EA01031843974B5860704798490866A4
:10112000704701460020934A506820F003000843AE
:10113000506070478F48406800F00C0070470146CF
:1011400000208C4A506820F0F0000843506070473F
:1011500001460020874A506820F4E0600843506050
:10116000704701460020834A506820F4605040EAEE
:10117000C1005060704729B17E4A527A02437D4BCC
:101180005A7204E07B4A527A82437A4B5A72704711
:101190007B49D8310860704701460020754A506885
:1011A00020F440400843506070470021714A2032CB
:1011B0001170704A82F82010012802D004280AD148
:1011C00004E001216B4A2032117005E00521694AD3
:1011D0002032117000E000BF00BF7047694908600D
:1011E00070476449096A0143624A11627047654960
:1011F00044390860704730B50021002200240023E4
:101200005C4D6D6805F00C0121B1042905D0082959
:1012100023D105E05C4D056022E05B4D05601FE0D9
:10122000544D6D6805F47012524D6D6805F48034AC
:10123000022505EB92421CB9544D554305600BE065
:101240004C4D6D6805F400351DB1504D554305609A
:1012500002E04D4D5543056002E04B4D056000BF77
:1012600000BF444D6D6805F0F0010909484D6B5C05
:101270000568DD4045603F4D6D6805F4E061090A91
:10128000434D6B5C4568DD4085603A4D6D6805F403
:101290006051C90A3E4D6B5C4568DD40C560354D07
:1012A0006D6805F44041890B3A4D6B5CC568B5FB30
:1012B000F3F5056130BD29B12E4A526902432D4B29
:1012C0005A6104E02B4A526982432A4B5A617047A3
:1012D00029B1284A92690243264B9A6104E0254AC3
:1012E00092698243234B9A61704729B1214AD2699E
:1012F0000243204BDA6104E01E4AD26982431D4B4F
:10130000DA61704729B11B4AD2680243194BDA608F
:1013100004E0184AD2688243164BDA60704729B15C
:10132000144A12690243134B1A6104E0114A12690C
:101330008243104B1A617047124940390860704768
:101340000F49C86470470B49C87170470948406A23
:1013500040F0807007494862704701460020054A06
:1013600092680A400AB1012000E00020704701495C
:1013700088727047001002400000FFF8FFFFF6FE81
:10138000000042428004424200127A0000093D00FF
:10139000140000202400002010B50446FE488442BA
:1013A00008D10121C014FFF7ADFF0021E014FFF7C1
:1013B000A9FFC4E0B4F1804F08D101210846FFF72E
:1013C000AEFF00210120FFF7AAFFB8E0F3488442F6
:1013D00008D101210220FFF7A2FF00210220FFF720
:1013E0009EFFACE0EE48844208D101210420FFF7C3
:1013F00096FF00210420FFF792FFA0E0E948844215
:1014000008D101210820FFF78AFF00210820FFF7FB
:1014100086FF94E0E448844208D101211020FFF7C0
:101420007EFF00211020FFF77AFF88E0DF4884422A
:1014300008D101212020FFF772FF00212020FFF7B3
:101440006EFF7CE0DA48844208D101214014FFF7A6
:1014500059FF00216014FFF755FF70E0D548844222
:1014600009D10121C804FFF74DFF00214FF40020EE
:10147000FFF748FF63E0D048844209D10121080505
:10148000FFF740FF00214FF48010FFF73BFF56E0CD
:10149000CA48844209D101214805FFF733FF0021E2
:1014A0004FF40010FFF72EFF49E0C548844208D1F1
:1014B00001214020FFF733FF00214020FFF72FFFDD
:1014C0003DE0C048844208D101218020FFF727FF7A
:1014D00000218020FFF723FF31E0BB48844208D180
:1014E00001218015FFF71BFF0021A015FFF717FF53
:1014F00025E0B648844209D101210804FFF702FF24
:1015000000214FF48030FFF7FDFE18E0B048844220
:1015100009D101214804FFF7F5FE00214FF4003006
:10152000FFF7F0FE0BE0AB48844208D101218804AC
:10153000FFF7E8FE00214FF48020FFF7E3FE10BD27
:1015400000220288944B98420ED0994B98420BD0BF
:10155000B0F1804F08D0914B984205D0904B984203
:1015600002D0904B984204D14FF68F731A404B88AB
:101570001A438D4B984207D08C4B984204D04FF6BB
:10158000FF431A40CB881A4302808B8883850B88DF
:101590000385814B98420BD0854B984208D08B4BEA
:1015A000984205D08A4B984202D08A4B984201D18A
:1015B0000B7A038601238382704770B500240022D2
:1015C0000023058C4FF6FE7635400584028C838817
:1015D000048B4FF68F752C40B51E2C400D882C4384
:1015E000751E2A400D892A434D882A436A4DA84218
:1015F0000BD06F4DA84208D0744DA84205D0744D51
:10160000A84202D0734DA84213D14FF6F7752A4075
:101610004D892A434FF6FB752A408D882A434FF6A1
:10162000FF652B404FF6FF552B408D892B43CD890D
:101630002B4383800483CD888586028470BD70B57A
:10164000002400220023058C4FF6EF7635400584F8
:10165000028C8388048B48F6FF752C404FF6FF45BB
:101660002C400D884FF6FF7606EA05252C434FF6F1
:10167000DF752A400D8906EA05152A434D8806EADA
:1016800005152A43444DA84202D0494DA8421DD118
:101690004FF67F752A404D894FF6FF7606EA05150D
:1016A0002A434FF6BF752A408D8806EA05152A435E
:1016B0004FF6FF352B404FF2FF752B408D8906EA20
:1016C00085052B43CD8906EA85052B43838004835A
:1016D000CD880587028470BD70B5002400220023E8
:1016E000058C4FF6FF6635400584028C8388848B19
:1016F0004FF68F752C404FF6FC752C400D882C430F
:101700004FF6FF552A400D894FF6FF7606EA05256C
:101710002A434D8806EA05252A431F4DA84202D0D8
:10172000234DA8421DD14FF2FF752A404D894FF637
:10173000FF7606EA05252A434FF6FF352A408D88B5
:1017400006EA05252A434EF6FF752B404DF6FF7538
:101750002B408D8906EA05152B43CD8906EA051530
:101760002B4383808483CD888587028470BD70B5C8
:10177000002200230024058C4EF6FF7635400584B8
:10178000038C8488828B48F6FF752A404FF6FF450C
:101790002A400D8820E00000002C01400004004099
:1017A00000080040000C0040001000400014004001
:1017B00000340140004C0140005001400054014001
:1017C00000180040001C0040002000400040014084
:1017D00000440140004801404FF6FF7606EA052527
:1017E0002A434DF6FF752B400D8906EA05352B433C
:1017F0004D8806EA05352B43FA4DA84202D0FA4D32
:10180000A84208D14BF6FF752C408D894FF6FF7624
:1018100006EA85152C4384808283CD88A0F8405049
:10182000038470BD828B4FF2FF331A408283828B18
:101830004FF6FF7303EA01231A4382837047F0B522
:101840000C461546002200210026078C4EF6FF7C30
:1018500007EA0C070784828B018C4FF6FF7707EAB3
:10186000043640F6FF473A404FF6FF7707EA052770
:101870003A434FF6FF7707EA03373A43D94FB84266
:101880000ED0D94FB8420BD0B0F1804F08D0D74F0F
:10189000B84205D0D64FB84202D0D64FB84206D192
:1018A0004DF6FF77394046F48057394305E047F657
:1018B000FF57394044F48057394382830184F0BD97
:1018C000828B4FF6F3731A408283828B0A438283A2
:1018D0007047F0B50C461546002200210026078C03
:1018E0004FF6FF6C07EA0C070784828B018C4FF6DA
:1018F000FF7707EA04264FF60C773A404FF6FF775A
:1019000007EA03172F433A43B64FB8420ED0B64FFB
:10191000B8420BD0B0F1804F08D0B44FB84205D0D8
:10192000B34FB84202D0B34FB84206D14FF6FF577B
:10193000394046F48077394305E04FF2FF5739408C
:1019400044F48077394382830184F0BD028B4FF2E7
:10195000FF331A400283028B4FF6FF7303EA012321
:101960001A4302837047F0B50C4615460022002149
:101970000026078C4FF6EF7C07EA0C070784028BE2
:10198000018C4FF6FF7707EA041640F6FF473A400E
:101990004FF6FF7707EA03373A434FF6FF7707EA38
:1019A00005273A438F4FB8420ED08F4FB8420BD025
:1019B000B0F1804F08D08D4FB84205D08C4FB8425F
:1019C00002D08C4FB84206D14FF6DF77394046F04F
:1019D0001007394305E04FF65F77394044F01007B0
:1019E000394302830184F0BD028B4FF6F3731A4032
:1019F0000283028B0A4302837047F0B50C461546FA
:101A000000220021068C4FF6FE773E400684028BB2
:101A1000018C4FF60C7632407E1C06EA03162E43EC
:101A20003243704EB0420ED06F4EB0420BD0B0F188
:101A3000804F08D06D4EB04205D06D4EB04202D0FE
:101A40006C4EB04206D14FF6FD76314044F00106AF
:101A5000314305E04FF6F576314044F0010631435D
:101A600002830184F0BD70B505460C465D48854291
:101A70000ED05D4885420BD0B5F1804F08D05B4851
:101A8000854205D05A48854202D05A48854200D145
:101A900000E000BF208850B92389A28861882846C9
:101AA000FFF7ABFFE1882846FFF79EFF25E020887F
:101AB00004280AD12389A28861882846FFF753FFAA
:101AC000E1882846FFF742FF17E0208808280AD15E
:101AD0002389A28861882846FFF7FBFEE188284613
:101AE000FFF7EEFE09E02389A28861882846FFF708
:101AF000A6FEE1882846FFF795FE70BD2DE9F0416E
:101B000005460C4600260127608808B9022600E039
:101B10000026A088012801D1022700E001272088A3
:101B2000A0B92389A28861882846FFF766FFE1886B
:101B30002846FFF759FF23893A4631462846FFF7E2
:101B400012FFE1882846FFF701FF13E02389A288EE
:101B500061882846FFF707FFE1882846FFF7F6FE71
:101B600023893A4631462846FFF747FFE188284651
:101B7000FFF73AFFBDE8F0810A884B881A438B884B
:101B80001A43CB881A430B891A434B891A438B8912
:101B90001A43A0F8442070474FF6FF71818000215E
:101BA0000180C18041800172704700210180418025
:101BB0008180C180018141818181C1817047002183
:101BC00001804180012181800021C1800181704715
:101BD0000021018041808180C1800181418181811A
:101BE00070470000002C0140003401400004004018
:101BF00000080040000C004021B1028842F00102C0
:101C0000028004E002884FF6FE731A40028070479B
:101C100031B1B0F8442042F40042A0F8442005E07D
:101C2000B0F84420C2F30E02A0F8442070471AB165
:101C300083890B43838102E083898B4383817047CF
:101C40008182704741EA0203A0F8483070471AB118
:101C500083890B43838102E083898B4383817047AF
:101C600001894FF6F8721140018170470A46002140
:101C700001894FF68F73194011430181704730B5C8
:101C800004460D4629462046FFF7F0FF208940F024
:101C90000700208130BD2DE9F04104460D4616466F
:101CA0001F46602D06D13B46012231462046FFF7F4
:101CB0005AFE05E03B46012231462046FFF79DFED5
:101CC00029462046FFF7D2FF208940F007002081F7
:101CD000BDE8F08130B50C4600210189C9B24FF64C
:101CE000FF7505EA0325154325432943018130BDCE
:101CF0002DE9F04105460E46174698460024434616
:101D00003A4631462846FFF7E5FF2C894FF6F87032
:101D1000044044F007044FF68F70044044F0700410
:101D20002C81BDE8F081F0B504460D4616461F46ED
:101D30003B46324629462046FFF7CCFF208940F437
:101D400080402081F0BD0185828270470A460021D3
:101D500001884FF68F731940114301807047F0B529
:101D60000C4615461E460021002200230189028BE5
:101D7000038C4FF6F877394021434FF6FC473A4041
:101D800040F201173A434FF6DD773B404FF6FF77BD
:101D900007EA06172F433B43018102830384F0BD0A
:101DA0000A460021018B4FF68F73194011430183BE
:101DB00070470A460021018B48F6FF7319404FF621
:101DC000FF7303EA02231943018370470A46002187
:101DD000818B4FF68F7319401143818370470A46F8
:101DE0000021818B48F6FF7319404FF6FF7303EA19
:101DF000022319438183704721B1028842F0800297
:101E0000028004E002884FF67F731A400280704718
:101E100021B1828842F00402828004E082884FF679
:101E2000FB731A408280704721B1828842F0080219
:101E3000828004E082884FF6F7731A4082807047F0
:101E400021B1828842F00102828004E082884FF64C
:101E5000FE731A40828070470A460021018B4FF6BC
:101E6000F77319401143018370470A460021018B23
:101E70004FF2FF7319404FF6FF7303EA0223194331
:101E8000018370470A460021818B4FF6F773194092
:101E90001143818370470A460021818B4FF2FF7303
:101EA00019404FF6FF7303EA0223194381837047F9
:101EB0000A460021018B4FF6FB7319401143018341
:101EC00070470A460021018B4FF6FF3319404FF649
:101ED000FF7303EA02231943018370470A46002176
:101EE000818B4FF6FB7319401143818370470A467B
:101EF0000021818B4FF6FF3319404FF6FF7303EA41
:101F000002231943818370470A460021018B4FF653
:101F10007F7319401143018370470A460021018BEA
:101F2000C1F30E014FF6FF7303EA02231943018345
:101F300070470A460021818B4FF67F731940114389
:101F4000818370470A460021818BC1F30E014FF651
:101F5000FF7303EA02231943818370470A46002175
:101F6000018C4FF6FD7319401143018470470A46F6
:101F70000021018C4FF6F77319401143018470471B
:101F80000A460021018C4FF6DF7319404FF6FF73AC
:101F900003EA02131943018470470A460021018CA9
:101FA0004FF67F7319404FF6FF7303EA021319438C
:101FB000018470470A460021018C4FF6FF531940F7
:101FC0004FF6FF7303EA02231943018470470A4660
:101FD0000021018C4FF2FF7319404FF6FF7303EAA3
:101FE00002231943018470470A460021018C4DF6F3
:101FF000FF7319404FF6FF7303EA0233194301845C
:10200000704730B5002301248C40A3B2048C9C435C
:102010000484048C02FA01F5ADB22C43048430BD73
:1020200030B5002304248C40A3B2048C9C43048468
:10203000048C02FA01F5ADB22C43048430BD70B5B6
:102040000346002000241846183001258D40ACB20C
:102050001D8CA5431D8409B1082909D100EB61003D
:10206000056825F0700505600568154305600EE0FC
:102070000D1FC5F34E052844056825F4E0450560AD
:1020800005684FF6FF7606EA02263543056070BD07
:1020900021B1028842F00202028004E002884FF679
:1020A000FD731A400280704721B1028842F0040299
:1020B000028004E002884FF6FB731A4002807047EA
:1020C00021B1828842F08002828004E082884FF64B
:1020D0007F731A408280704702884FF6F7731A4068
:1020E000028002880A430280704782884FF68F730D
:1020F0001A40828082880A438280704702894FF6A4
:10210000F8731A40028102890A43028170470289EA
:102110004FF67F731A40028102890A430281704799
:102120008184704781857047818670470187704739
:1021300081877047A0F84010704702884FF6FF4330
:102140001A40028002880A43028070470146888E46
:1021500070470146088F70470146888F70470146D7
:10216000B1F8400070470146888C70470146088DE1
:10217000704702460020138A0B400BB1012000E09B
:1021800000207047CA430282704730B502460020E3
:1021900000230024158A05EA0103958905EA010454
:1021A00013B10CB1012000E0002030BDCA4302820F
:1021B0007047000010B50446FB48844209D1012154
:1021C0008803FFF79FF800214FF48040FFF79AF84B
:1021D00032E0F648844209D101214804FFF79FF814
:1021E00000214FF40030FFF79AF825E0F0488442D0
:1021F00009D101218804FFF792F800214FF48020D3
:10220000FFF78DF818E0EB48844209D10121C8049A
:10221000FFF785F800214FF40020FFF780F80BE06E
:10222000E548844208D101210805FFF778F800212C
:102230004FF48010FFF773F810BD2DE9F04786B01A
:1022400005460E460024A24600BFA1460027B089DD
:1022500000B100BF2F462C8A4CF6FF700440F08876
:1022600004432C82AC894EF6F3100440B0883189C7
:102270000843718908430443AC81AC8A4FF6FF40A0
:102280000440B0890443AC8201A8FEF7B4FFC648FD
:10229000874202D1DDF810A001E0DDF80CA0A8898A
:1022A00000F4004040B10AEBCA0000EB0A103168AC
:1022B0004900B0FBF1F807E00AEBCA0000EB0A1096
:1022C00031688900B0FBF1F86420B8FBF0F004013C
:1022D0002009642101FB1089A88900F4004040B165
:1022E000322000EBC900B0FBF1F000F0070004431E
:1022F00008E0322000EB09106421B0FBF1F000F09F
:102300000F0004432C8106B0BDE8F0874FF416514E
:10231000016000218180C18001810C214181002167
:102320008181704710B502460020108A4FF2FF03EA
:1023300018400B884C8823438C882343CC88234344
:102340001843108210BD0021018041808180C1802E
:10235000704721B1828942F40052828104E082896F
:102360004DF6FF731A4082817047F0B50346002492
:1023700000260025002040F66A17B94200D100BFB0
:102380001846C1F3421401F01F06012707FA06F5AB
:10239000012C01D10C3004E0022C01D1103000E0FE
:1023A00014301AB107682F43076002E00768AF4393
:1023B0000760F0BD1AB1838A0B43838202E0838AEF
:1023C0008B4383827047028A4FF6F0731A40028271
:1023D000028A0A430282704782894FF2FF731A40D1
:1023E000828182890A438281704721B1828942F0C9
:1023F0000202828104E082894FF6FD731A408281D5
:102400007047028A4FF6DF731A400282028A0A433B
:102410000282704721B1028A42F48042028204E0C3
:10242000028A4BF6FF731A4002827047C1F308021A
:102430008280704701468888C0F308007047818910
:1024400041F0010181817047028BD2B20283028B7D
:1024500042EA012202837047028B02F47F42028328
:10246000028B0A430283704721B1828A42F0200224
:10247000828204E0828A4FF6DF731A4082827047BC
:1024800021B1828A42F01002828204E0828A4FF6F1
:10249000EF731A408282704721B1828A42F00802AB
:1024A000828204E0828A4FF6F7731A408282704774
:1024B00021B1828942F40042828103E08289C2F321
:1024C0000E028281704721B1828A42F400628282C8
:1024D00004E0828A4FF2FF731A4082827047828A38
:1024E0004FF6FB731A408282828A0A4382827047C7
:1024F00021B1828A42F00202828204E0828A4FF68F
:10250000FD731A408282704702460020B1F5007FB9
:1025100000D100BF13880B400BB1012000E0002068
:10252000704701F40072B2F5007F00D100BFCA43CA
:102530000280704770B50246002400230025002069
:1025400040F66A16B14200D100BFC1F3421501F056
:102550001F03012606FA03F3012D02D196893340A9
:1025600006E0022D02D1168A334001E0968A3340FC
:102570000C12012606FA04F41688344013B10CB18B
:10258000012000E0002070BD10B50022002340F6BD
:102590006A14A14200D100BF0A1201249440A3B2E0
:1025A000DC43048010BD00000038014000440040BE
:1025B00000480040004C004000500040094880475F
:1025C00009480047FEE7FEE7FEE7FEE7FEE7FEE715
:1025D000FEE7FEE7FEE7FEE704480549054A064B2D
:1025E00070470000C1040008ED000008E001002071
:1025F000E0070020E0030020E003002008B50121EF
:102600000C20FEF765FE0120ADF8000010208DF8CB
:10261000030003208DF8020069460848FEF77CFBA2
:102620000120ADF8000010208DF8030003208DF884
:10263000020069460248FEF76FFB08BD000C01402E
:102640000008014070B505460C4645F25550FEF7AE
:10265000B1FC2846FEF7B1FC2046FEF7B1FCFEF7C0
:10266000B2FCFEF7B5FC70BD10B5FEF7ACFC10BDBA
:102670007FB505460C4601210220FEF736FEADF877
:102680000850ADF804400020ADF80A00ADF806008F
:1026900001A93848FEF754FF012211463548FFF7DB
:1026A000C6FA1D208DF8000000208DF801000320DF
:1026B0008DF8020001208DF803006846FDF785FFC4
:1026C00000212C48FFF798FA7FBD7FB505460C46E0
:1026D00001210420FEF709FEADF80850ADF80440D2
:1026E0000020ADF80A00ADF8060001A92248FEF767
:1026F00027FF012211462048FFF799FA1E208DF886
:10270000000003208DF801008DF8020001208DF8F3
:1027100003006846FDF759FF01211748FFF76CFADF
:102720007FBD10B501211348FFF72FFDA8B101218E
:102730001048FFF73BFD11480078401C0F49087016
:10274000084600781E2808DB0020087001200C498C
:10275000087000210748FFF74FFA10BD10B501219E
:102760000548FFF712FD18B101210348FFF71EFDD0
:1027700010BD0000000400400008004028000020B8
:102780002900002010B5DB4800F031FD002404E0F2
:102790000020D8490855601CC4B2642CF8DB002026
:1027A000D5490870FFF760FF10BD10B5D3A000F049
:1027B00087FD4FF4967000F0CCFBD2A1CD4800F01D
:1027C000B5FFD1490860FFF7DDFF0EE0FFF7DAFF44
:1027D000CAA000F075FD4FF4967000F0BAFBC9A1D5
:1027E000C44800F0A3FFC8490860C7480068002833
:1027F000ECD0C6A000F064FD4FF4967000F0A9FB89
:10280000C5A000F05DFD4FF4967000F0A2FBC5A1DD
:10281000B84800F08BFFBC490860FFF7B3FF0EE03B
:10282000FFF7B0FFBCA000F04BFD4FF4967000F036
:1028300090FBBCA1AF4800F079FFB3490860B248F3
:1028400000680028ECD0B8A000F03AFD4FF4967074
:1028500000F07FFBABA1A74800F068FFAA49086021
:10286000FFF790FFB4A000F02BFD4FF4967000F03E
:1028700070FBB4A19F4800F059FFA3490860FFF71F
:1028800081FF0EE0FFF77EFFABA000F019FD4FF4D3
:10289000967000F05EFBABA1964800F047FF9A49A6
:1028A0000860994800680028ECD0A9A000F008FD55
:1028B0004FF4967000F04DFBA8A18E4800F036FF53
:1028C000914908600846006830B308460068007AFD
:1028D00030380968C979303901EB810100EB4100DA
:1028E000A049087008460078632804D0864800682C
:1028F000C079303860B90AE000209A4981F8720046
:1029000099A000F074FC4FF4967000F022FBF3E7FE
:102910000120944981F87200FFF734FF10BD10B513
:1029200098A000F0CDFC4FF4967000F012FBFFF77A
:1029300029FFFFF799FE10BD10B596A000F0C0FC6E
:102940004FF4967000F005FB9FA16A4800F0EEFE80
:102950006D49086008E09CA1664800F0E7FE6A49FE
:102960000860642000F0F5FA674800680028F2D09B
:10297000FFF708FF10BD70B504460D462A462146F4
:1029800095A000F09DFC70BD70B504460D462A462A
:10299000214697A000F094FC4FF4967000F0D9FA0D
:1029A00008E099A1534800F0C1FE5749086064202F
:1029B00000F0CFFA544800680028F2D0FFF7E2FE9A
:1029C00070BD704710B592A39AA29CA19EA000F082
:1029D00077FC4FF4967000F0BCFAA5A000F070FCF4
:1029E0004FF4967000F0B5FAABA1424800F09EFE9D
:1029F0004549086005E0A8A13E4800F097FE42491D
:102A00000860414800680028F5D0FFF7BBFEA6A08B
:102A100000F056FC4FF4967000F09BFAABA13548DD
:102A200000F084FE3849086005E0A8A1314800F0B4
:102A30007DFE35490860344800680028F5D0FFF76E
:102A4000A1FE10BDF0B5D7B007460C461546902242
:102A5000A24933A800F0E0FE2B46224633A901A884
:102A600000F03AFC01A800F073FE86B2324601A9DC
:102A7000384600F08CFEF0B257B0F0BD70B5B2B081
:102A800004460D4696A1A3A000F01AFC4FF49670E0
:102A900000F05FFA2A4621466846FFF7D3FF064654
:102AA00000200DF806006946A0A000F009FC00BF58
:102AB0009F48008800F040000028F9D01A209C4967
:102AC000091D0880642000F044FA9AA1094800F02A
:102AD0002DFE0D49086005E096A1064800F026FE8F
:102AE00009490860084800680028F5D0FFF74AFE49
:102AF00032B070BDB70000204000002041540D0AE4
:102B0000000000004F4B00002C00002041542B43DC
:102B100046554E3D310D0A0041542B43494D490D58
:102B20000A0000003436300041542B4347415454CE
:102B30003D310D0A0000000041542B4347415454DD
:102B40003F0D0A002B43474154543A203100000006
:102B500041542B434553510D0A0000002B4345536C
:102B60005100000044000020D0C5BAC5CBD1CBF73E
:102B7000CAA7B0DCA3ACC7EBB2E9BFB4D4ADD2F204
:102B8000210D0A0041542B5149434C4F53453D30D0
:102B90000D0A000041542B51494F50454E3D312CF8
:102BA000302C22544350222C2234372E39392E38DF
:102BB000302E3839222C31343236392C31323334FC
:102BC0002C310D0A000000002B51494F50454E3A60
:102BD00020302C300000000041542B51534F5345FE
:102BE0004E443D302C25732C25730D0A0000000047
:102BF00041542B514953454E4445583D302C257383
:102C00002C25730D0A00000053454E44204F4B0005
:102C10007A50776F4A467153455343446775634909
:102C20004B346C4B76786546715556463773427512
:102C3000000000006D7A68303032000061314E587B
:102C40006F7865467734630041542B514D544346A9
:102C5000473D22616C6961757468222C302C2225F5
:102C600073222C222573222C222573220D0A0000A8
:102C700041542B514D544F50454E3D302C22313351
:102C8000392E3139362E3133352E313335222C3130
:102C90003838330D0A0000002B514D544F50454E2B
:102CA0003A20302C3000000041542B514D54434FFA
:102CB0004E4E3D302C22636C69656E744578616DB3
:102CC000706C655F31393837220D0A002B514D5435
:102CD000434F4E4E3A20302C302C3000B03B000891
:102CE0002F7379732F61314E586F7865467734634F
:102CF0002F6D7A683030322F7468696E672F657671
:102D0000656E742F70726F70657274792F706F7347
:102D10007400000041542B514D545055423D302C0D
:102D2000302C302C302C25730D0A00002573000048
:102D3000004400402B514D545055423A20302C3025
:102D40002C30000010B56048006820F0F0005E49AB
:102D500008600846006840F03000086000205B49C9
:102D60000860142000F0F5F801205949C1F88401E9
:102D70001E2000F0CAF810BD10B5002452480068AB
:102D800020F0F000504908600846006840F08000DC
:102D9000086004E0601CC4B2012000F0B6F84B48A3
:102DA0008038006808B1642CF4DB642C01DB01205E
:102DB00010BD002404E0601CC4B2012000F0A5F89E
:102DC00042488038006808B9642CF4DB642C01DBCD
:102DD0000120EDE70020EBE710B5002404E0601CC3
:102DE000C4B2012000F091F838488038006808B17A
:102DF000642CF4DB002404E0601CC4B2012000F069
:102E000084F832488038006808B9642CF4DB282044
:102E100000F07BF82D488038006808B1012010BD13
:102E20000020FCE770B50024002506E06006040ED3
:102E3000FFF7D2FF0443681CC5B2082DF6DB20461D
:102E400070BD7CB505460E46FFF77CFFFFF794FF8B
:102E5000F8B9002405E0FFF7E5FF0DF80400601C59
:102E6000C4B2052CF7DB9DF800009DF80110084462
:102E70009DF8021008449DF8031008449DF80410C2
:102E8000884208D19DF8000030709DF8020028703B
:102E900001E001207CBD0020FCE710B50D488069F1
:102EA00040F008000B4988610748006820F0704036
:102EB000054908600846006840F030000860FFF7E8
:102EC00041FFFFF759FF10BD000C014084812142F2
:102ED000008021420010024010B56FF00400FDF7A1
:102EE000BEFB2E4800682E49B0FBF1F02D4908705A
:102EF0000846007800EB4001C1EBC0104FF6FF71AF
:102F000001EAC0002849088010BD0146254A127810
:102F10004A434FF0E0235A6100229A611A4612692F
:102F200042F001021A6100BF4FF0E022106900F088
:102F300001021AB100F48032002AF5D04FF0E022ED
:102F4000126922F001024FF0E0231A6100229A6117
:102F500070470146144A12884A434FF0E0235A61F1
:102F600000229A611A46126942F001021A6100BFFA
:102F70004FF0E022106900F001021AB100F4803233
:102F8000002AF5D04FF0E022126922F001024FF042
:102F9000E0231A6100229A617047000000000020BF
:102FA00000127A00340000203600002010B54FF4E3
:102FB000A060FDF705FB10BD00BF704700BFB84A19
:102FC000128802F04002002AF9D0C2B2B44B1B1D95
:102FD0001A80704710B5044600BF8021B148FFF742
:102FE00093FA0028F9D02146AE48FFF71FFA10BD2A
:102FF00010B5044600BF8021A948FFF785FA0028D4
:10300000F9D02146A648FFF711FA10BD10B586B0D9
:103010000446012144F20400FEF75AF9A148FFF7E3
:10302000C9F84FF40070ADF8140003208DF81600B5
:1030300018208DF8170005A99B48FDF76DFE4FF489
:103040008060ADF8140048208DF8170005A9964857
:10305000FDF762FE25208DF8000003208DF80100A9
:103060008DF8020001208DF803006846FDF7ADFAE7
:1030700001940020ADF80800ADF80A00ADF80C008E
:10308000ADF810000C20ADF80E0001A98548FFF73F
:10309000D4F8012240F225518248FFF766F9012158
:1030A0008048FFF756F906B010BD10B586B004464B
:1030B00001210420FEF70CF901214804FEF715F95F
:1030C0007748FFF777F80420ADF8140003208DF857
:1030D000160018208DF8170005A97348FDF71CFE8F
:1030E0000820ADF8140004208DF8170005A96E48DB
:1030F000FDF712FE26208DF8000000208DF801005B
:1031000001208DF802008DF803006846FDF75DFA96
:1031100001940020ADF80800ADF80A00ADF80C00ED
:10312000ADF810000C20ADF80E0001A95C48FFF7C7
:1031300084F8012240F225515948FFF716F9012180
:103140005748FFF706F906B010BD10B586B0044623
:1031500001210820FEF7BCF801218804FEF7C5F81C
:103160005248FFF727F84FF48060ADF814000320B1
:103170008DF8160018208DF8170005A94C48FDF7AA
:10318000CBFD4FF40060ADF8140004208DF817005B
:1031900005A94748FDF7C0FD27208DF80000002055
:1031A0008DF8010001208DF802008DF803006846BB
:1031B000FDF70BFA01940020ADF80800ADF80A0005
:1031C000ADF80C00ADF810000C20ADF80E0001A910
:1031D0003648FFF732F8012240F225513348FFF715
:1031E000C4F801213148FFF7B4F806B010BD0BE078
:1031F00000BF2C49098801F040010029F9D001786D
:10320000284A121D1180401C01780029F0D1704716
:103210000BE000BF2549098801F040010029F9D0E1
:103220000178224A121D1180401C01780029F0D13A
:10323000704710B540F225511A48FFF77BF918B1D5
:103240001848FFF7F7F8C4B210BD10B540F2255189
:103250001348FFF76FF9B0B11148FFF7EBF8C4B2AC
:103260000F48FFF7E7F8C1B2124802780078401C17
:10327000104B18701048815418460078632802DDFE
:1032800000201946087010BD10B540F225510748BE
:10329000FFF750F918B10548FFF7CCF8C4B210BDDC
:1032A0000044004000380140000801400048004050
:1032B000000C014040000020B700002070470000D3
:1032C0000FB4044910B503AA029800F069FB10BCC2
:1032D0005DF814FB3C0000200FB41CB5074B06AA98
:1032E0007B4469460090059800F02BFB002069465E
:1032F00000F03AFB1CBC5DF814FB000085060000E2
:1033000070B5044685690068C10601D5302600E025
:103310002026C00707D070BDD4E901213046904770
:10332000206A401C20626D1EF6D570BD70B5044643
:1033300085690078C00707D170BDD4E9012120203C
:103340009047206A401C20626D1EF6D570BD09684A
:103350004A0501D540B27047C905FCD500B2704797
:1033600009684A0501D5C0B27047C905FCD580B2CD
:10337000704770B50C460546012A05D028788006AE
:1033800000D5EA69002302E0012305E05B1C9342BB
:1033900002D2E05C0028F9D1A869E618C01AA86139
:1033A000286A184428622846FFF7AAFF04E0D5E9F6
:1033B000012114F8010B9047B442F8D32846FFF7D7
:1033C000B5FF70BD2DE9F04106460024106875294F
:1033D000314616A510D0FFF7BAFF002802DA4042A6
:1033E00013A507E031688A0701D512A502E0490755
:1033F00004D511A5012401E0FFF7B2FF00210A2244
:1034000006F1240709E0B0FBF2FCB0FBF2F302FB8B
:103410001C00303078541846491C0028F3D123464C
:103420002A463046BDE8F04100F02CBA000000000A
:103430002D0000002B000000200000002DE9FF5FA0
:1034400015468A460446DFF8AC80F8440027D8E9E0
:1034500000103E46CDE9001010E03AF816106A461A
:1034600002A800F0C5FA411C07D02178890603D5CF
:10347000E269391891420DD80744761C20788006FD
:1034800002D5E069B84205DDAE42E6DB3AF8160047
:103490000028E2D1A069C01BA0612046FFF730FFE1
:1034A000D8E90010CDE90010002017E03AF8181014
:1034B0006A4602A800F09CFAB0F1FF3F81460BD0AB
:1034C00000250DF1080B05E0D4E901211BF80500EA
:1034D00090476D1C4D45F7D308F10100B04280467E
:1034E000E4DB206A384420622046FFF71FFFBDE876
:1034F000FF9F00001E07000070B5044621461068BB
:10350000FFF72EFF002104F1240505E000F007027B
:103510003032C0086A54491C0028F7D120680023C3
:1035200008A2050708D500F02000084304D0E06990
:10353000012305A2401EE0612046BDE8704000F076
:10354000A1B90000000000003000000070B5044682
:103550000D4621461068FFF703FF2188090502D5B3
:103560000F4A7A4402E00E4A7A440E32002104F1F6
:10357000240305E000F00F060009965D5E54491C27
:103580000028F7D120780023000704D5702D02D041
:1035900009B1022311322046BDE8704000F072B933
:1035A0000E0600002DE9F05F894604464FF0000A40
:1035B000DFF874B1FB44C0F820A02046E1688847DA
:1035C000002874D0252806D0D4E901219047206A2C
:1035D000401C2062F1E700265F462046E1688847EC
:1035E0002028054607DB312D05D2781910F8200C6C
:1035F00008B10643F1E7B00701D526F00406C4F888
:103600001CA00027C4F818A02A2D09D0284600F0D5
:103610008FFA38B304EB8708303DC8F8185019E02A
:1036200059F8041B204604EB87029161E168884742
:10363000012F054618D1E069002820DA26F020067F
:103640001DE0D8F8180000EB800005EB4000303892
:10365000C8F818002046E1688847054600F068FA77
:103660000028EED1012F0AD02E2D08D12046E16886
:1036700088477F1C0546022F46F02006C4DBA06960
:10368000002803DA404246F00106A061F00701D0AD
:1036900026F010066C2D0BD0682D09D04C2D39D09A
:1036A0006A2D35D0742D35D07A2D33D016E038E020
:1036B000E1682F4620468847B842054609D16C2F5D
:1036C00026D04FF48060E1680643204688470546CF
:1036D00004E06C2F1AD04FF4807006430DB3A5F1AF
:1036E0004100192802D8203546F400664A4629468A
:1036F000204626604E46FCF733FD80B101280BD0F2
:10370000F61D26F0070000F1080956E74020E4E71F
:103710008020D8E70020D6E706F104094DE72846C7
:1037200052E7206ABDE8F09FE405000030B5054689
:103730000B462A4613F8014B12F8010B08B1A042C0
:10374000F8D01CB1002802D06D1CF1E7284630BD2E
:1037500010B5431C02E010F8011B71B18107FAD1CA
:103760004FF0013202C88C1A8C4314EAC211F9D00E
:10377000C01A0A0603D0C01E10BDC01A10BD0A042C
:1037800001D0801E10BD0902FCD0401E10BD032ACE
:1037900040F2308010F0030C00F0158011F8013B6E
:1037A000BCF1020F624498BF11F801CB00F8013B55
:1037B00038BF11F8013BA2F1040298BF00F801CB19
:1037C00038BF00F8013B11F0030300F02580083AF0
:1037D000C0F0088051F8043B083A51F804CBA0E847
:1037E0000810F5E7121D5CBF51F8043B40F8043B9C
:1037F000AFF30080D20724BF11F8013B11F801CBD1
:1038000048BF11F8012B24BF00F8013B00F801CBA1
:1038100048BF00F8012B704710B5203AC0F00B806C
:10382000B1E81850203AA0E81850B1E81850A0E8C4
:103830001850BFF4F5AF5FEA027C24BFB1E818501E
:10384000A0E8185044BF18C918C0BDE810405FEA8E
:10385000827C24BF51F8043B40F8043B08BF70470A
:10386000D20728BF31F8023B48BF11F8012B28BF0F
:1038700020F8023B48BF00F8012B704770477047A3
:10388000704770472DE9F0470D4699469246044629
:1038900000F124080168880604D5E06921F01001D0
:1038A000216000E00120A84201DD471B00E0002765
:1038B000A1697A1902EB0900081AA0612078C006F4
:1038C00002D42046FFF71CFD002608E0D4E90121C0
:1038D0001AF806009047206A401C761C20624E456C
:1038E000F4DB2078C0060AD52046FFF709FD06E084
:1038F000D4E9012130209047206A401C2062381E04
:10390000A7F10107F4DC07E0D4E9012118F805006C
:103910009047206A401C2062281EA5F10105F3DCB7
:103920002046FFF703FD2078000602D50220BDE8FF
:10393000F0870120FBE7000001694A1C026108785A
:10394000704700B58FB0CDE90131002105910549DF
:103950007944CDE9031011466846FFF723FE0FB006
:1039600000BD0000E5FFFFFF0A6802F8010B0A60D6
:10397000704710B5436913B1AFF3008001E0FFF762
:10398000F8FC012010BD127800F124010A70002219
:103990004A700122EDE711684FF0FF32E9E70000BD
:1039A000074B70B50D467B44FFF7CBFF0446284616
:1039B00000F046F810B14FF0FF3070BD204670BDEA
:1039C00013F6FFFF10B5436913B1AFF3008001E0B8
:1039D000FFF734FD012010BD128800F1240182841C
:1039E0000022C2840122EDE711684FF0FF32E9E7BF
:1039F00070B516460C46054600F01AF8036893F8B1
:103A00000101012806D0FF2C0FD8185D68B10120F4
:103A10002C7070BDD3F807013246214603F207131C
:103A200003442846BDE8704018474FF0FF3070BD92
:103A300010B500F02FF8001D10BD00BF05010000FB
:103A4000007B00F080007047754600F02DF8AE4610
:103A500005006946534620F00700854618B020B59A
:103A6000FEF7BAFDBDE820404FF000064FF000071A
:103A70004FF000084FF0000B21F00701AC46ACE816
:103A8000C009ACE8C009ACE8C009ACE8C0098D4683
:103A90007047000000487047A00100200446AFF3C3
:103AA00000802046FCF791FB004870478001002011
:103AB0004FF0013C50F8042B51F8043B9A4221D1BD
:103AC000A2EB0C03934313EACC1317D150F8042B49
:103AD00051F8043B9A4215D1A2EB0C03934313EA2D
:103AE000CC130BD150F8042B51F8043B9A4209D166
:103AF000A2EB0C03934313EACC13DBD04FF000008E
:103B0000704700BFD01A01BAB1FA81F101F0180173
:103B100022FA01F0CB40C1F12001DBB2C0B2C01AE1
:103B20002CFA01F3D11A914311EAC311E6D170477F
:103B300030380A2801D20120704700207047000069
:103B400010B500290AD00878002807D00548784425
:103B5000FFF7AEFF002801D0002010BD02487844D6
:103B600010BD0000120100000A010000000000006A
:103B700000000000303132333435363738394142B5
:103B800043444546403058003031323334353637BF
:103B9000383961626364656640307800040000086B
:103BA0000000000000000002000100001000000002
:103BB0007B226964223A223236222C227665727385
:103BC000696F6E223A22312E30222C22706172618E
:103BD0006D73223A7B2243757272656E7454656D03
:103BE0007065726174757265223A7B2276616C75BC
:103BF00065223A25647D2C2252656C617469766574
:103C000048756D6964697479223A7B2276616C75B6
:103C100065223A25647D7D2C226D6574686F64226F
:103C20003A227468696E672E6576656E742E7072BE
:103C30006F70657274792E706F7374227D0000004E
:103C4000703D00080000002044000000280100082A
:103C5000B43D0008440000209C0700004401000817
:103C60001001000043000000F8FFFFFF004040404B
:103C7000404040404040414141414140404040403F
:103C800040404040404040404040404040050202EB
:103C900002020202020202020202020202202020AA
:103CA0002020202020202002020202020202909006
:103CB0009090909010101010101010101010101004
:103CC0001010101010101010020202020202888858
:103CD0008888888808080808080808080808080864
:103CE000080808080808080802020202400000004C
:103CF00000000000000000000000000000000000C4
:103D000000000000000000000000000000000000B3
:103D100000000000000000000000000000000000A3
:103D20000000000000000000000000000000000093
:103D30000000000000000000000000000000000083
:103D40000000000000000000000000000000000073
:103D50000000000000000000000000000000000063
:103D60000000000000000000000000000000000053
:103D700000A24A0400000000000000000102030449
:103D80000607080900000000010203040102030401
:103D900006070809020406080000000000000000F1
:103DA0000000000000000000000000000000000013
:043DB000000000000F
:04000005080000ED02
:00000001FF
